:020000040000FA
:040000006C303A28FE
:08000800A000030EA100831209
:100010008B1C32288B1031181428B11C3228643004
:10002000010203183128182800001628172818285C
:1000300019281A281B281C281D281E281F283110A3
:10004000B114A810031005190314AA0DA90DA80DC9
:10005000B00B322831152A08AF002908AE00280855
:10006000AD00B11081010B11210E8300A00E200EF6
:02007000090085
:0C007400203084008001840A6030040207
:10008000031C3C281230B0009A218316FF239000F5
:10009000831283160C308505870183128501870141
:1000A000073099000030831691008312C830831600
:1000B0008100831231309000003083168C0083124F
:1000C00010308B00831600309B001C141A0883121A
:1000D000BC00851DDE21831610309B001C141A08FD
:1000E0008312BD00D62181018E018F010B118B106F
:1000F0000B108C018B178A203119A020B30B882894
:10010000031085190314B90DF030390203191921B0
:1001100003227B286400311808000B1D08000B1116
:10012000B11031141230B000051D9B283214831613
:10013000011383120800321083160117831208007E
:1001400031110130B7008B132030370783169B0025
:100150001C141A088312A400A500C030A506103094
:10016000370783169B001C141A088312A300003063
:10017000370783169B001C141A088312A2008B17E2
:10018000321CC82822090339A200A309A409A50921
:1001900022082D02031D132923082E02031D1329F3
:1001A00024082F02031D132901303702031DDD2807
:1001B0003D18DD283D143E14A62102303702031DF0
:1001C000E628BD18E628BD143E14A82103303702E6
:1001D000031DEF283D19EF283D153E14AA210430D8
:1001E0003702031DF828BD19F828BD153E14AC21AF
:1001F00005303702031D01293D1A01293D163E1421
:10020000AE2106303702031D0A29BD1A0A29BD1680
:100210003E14B02107303702031D13293D1B13295B
:100220003D173E14B221B70A083037020318080000
:10023000A3280130B600B300B400B500B7008501B3
:100240008701B1138A20B30B4D29031085190314BC
:10025000B90DF030390203197429B40B4D2901305E
:1002600037020319BD21023037020319C2210330BE
:1002700037020319C521043037020319C82105309C
:1002800037020319CD21063037020319D021073078
:1002900037020319D3219630B400311D22293111C0
:1002A000321C57292D090339AD00AE09AF092F1CA7
:1002B000B1132F1C2229B11B22292E182229B11774
:1002C0008B1320303707BB002F08BA00872110306E
:1002D0003707BB002E08BA00872100303707BB0064
:1002E0002D08BA0087218B1785018701B70AB6014F
:1002F00008303702031C2229D62108003E1C0800C2
:100300003E101030BB003D08BA00872108008B1357
:100310003A0883161C159A003B089B0055309D0037
:10032000AA309D009C1464009C1893291C11831210
:100330008B170800FF30D000D415D515D615D7156A
:10034000D815D915DA15DB15DC150800F130B529FB
:10035000F230B529F430B529F830B5291F30B92964
:100360002F30B9294F30B9290800BD050F30D2040C
:100370000800BD05F030D2040800103085060230B8
:100380008706080020308506080021308506080011
:1003900002308506023087060800183087060800FC
:1003A0002130870608000930870608003D08D20082
:1003B000031D08001130BD00D2000800B601B301D2
:1003C000B4013C1CE629BC01BC14E829BC013C1466
:1003D0003C08B6006400EC29ED29EE29EF29F0294C
:1003E000B41B0516B41F0512B30BEA29B40BEA2996
:1003F0000310B60CB608031DEA290030BB003C0808
:10040000BA00872108008F08031908008F01D00F58
:100410003E2BD00A0E305205031D1D2A541D132AEF
:10042000D40154162B2AD41D182AD40154162B2A71
:10043000541E2B2AD401D4142B2AD41C222AD401D2
:1004400054152B2A541D272AD401D4152B2A541EA7
:100450002B2AD401541509305205031D3E2A551D7F
:10046000342AD50155164C2AD51D392AD5015516E1
:100470004C2A551E4C2AD501D5144C2AD51C432A8A
:10048000D50155154C2A551D482AD501D5154C2A9C
:10049000551E4C2AD50155150B305205031D5F2AF8
:1004A000561D552AD60156166D2AD61D5A2AD60132
:1004B00056166D2A561E6D2AD601D6146D2AD61CE4
:1004C000642AD60156156D2A561D692AD601D615FD
:1004D0006D2A561E6D2AD601561507305205031D8A
:1004E000802A571D762AD70157168E2AD71D7B2AB8
:1004F000D70157168E2A571E8E2AD701D7148E2A57
:10050000D71C852AD70157158E2A571D8A2AD7014D
:10051000D7158E2A571E8E2AD70157150630520539
:10052000031DA12A581D972AD8015816AF2AD81D95
:100530009C2AD8015816AF2A581EAF2AD801D814C1
:10054000AF2AD81CA62AD8015815AF2A581DAB2AA5
:10055000D801D815AF2A581EAF2AD8015815103027
:10056000BC1819305205031DC42A591DBA2AD901D5
:100570005916D22AD91DBF2AD9015916D22A591E75
:10058000D22AD901D914D22AD91CC92AD90159157C
:10059000D22A591DCE2AD901D915D22A591ED22ABA
:1005A000D90159155030BC1859305205031DE72A9E
:1005B0005A1DDD2ADA015A16F52ADA1DE22ADA0175
:1005C0005A16F52A5A1EF52ADA01DA14F52ADA1C27
:1005D000EC2ADA015A15F52A5A1DF12ADA01DA1540
:1005E000F52A5A1EF52ADA015A156030BC1869300E
:1005F0005205031D0A2B5B1D002BDB015B16182B1C
:10060000DB1D052BDB015B16182B5B1E182BDB019A
:10061000DB14182BDB1C0F2BDB015B15182B5B1D70
:10062000142BDB01DB15182B5B1E182BDB015B1574
:100630002030BC1829305205031D2D2B5C1D232BA7
:10064000DC015C163B2BDC1D282BDC015C163B2BF4
:100650005C1E3B2BDC01DC143B2BDC1C322BDC0155
:100660005C153B2B5C1D372BDC01DC153B2B5C1E2A
:100670003B2BDC015C157E213D08D2005008D100E7
:100680000C305405031D05120C305505031D851251
:100690000C305605031D05100C305705031D851041
:1006A0000C305805031D87100C305905031D071029
:1006B0000C305A05031D87120C305B05031D071211
:1006C0000C305C05031D871151080E020318902B96
:1006D00012305405031D051612305505031D8516ED
:1006E00012305605031D051412305705031D8514DD
:1006F00012305805031D871412305905031D0714C5
:1007000012305A05031D871612305B05031D0716AC
:1007100012305C05031D8715FF30500203190800D5
:100720008F08031D08008A2051080E02031C902B1D
:1007300018305405031D051206305405031D051617
:1007400018305505031D851206305505031D851605
:1007500018305605031D051006305605031D0514F7
:1007600018305705031D851006305705031D8514E5
:1007700018305805031D871006305805031D8714CF
:1007800018305905031D071006305905031D0714BD
:1007900018305A05031D871206305A05031D8716A7
:1007A00018305B05031D071206305B05031D071695
:1007B00018305C05031D871106305C05031D871585
:0207C00008002F
:084000000A00030002000600A3
:02400E00CC01E3
:10420000010003000300030003000200020002009B
:1042100002000000000000000000FF00FF00FF009F
:10422000000000000000000000000000000000008E
:104230000000C000C000C000C000FF00FF00FF0081
:104240000100C300F300CF00FF00C300F300CF0064
:10425000FF00C300F300CF00FF00FF00FF00FF00DE
:10426000FF00FF00FF00FF00FF00FF00FF00FF0056
:10427000FF00FF00FF00FF00FF00FF00FF00FF0046
:10428000FF00FF00FF00FF00FF00FF00FF00FF0036
:10429000FF00FF00FF00FF00FF00FF00FF00FF0026
:1042A000FF00FF00FF00FF00FF00FF00FF00FF0016
:1042B000FF00FF00FF00FF00FF00FF00FF00FF0006
:1042C000FF00FF00FF00FF00FF00FF00FF00FF00F6
:1042D000FF00FF00FF00FF00FF00FF00FF00FF00E6
:1042E000FF00FF00FF00FF00FF00FF00FF00FF00D6
:1042F000FF00FF00FF00FF00FF00FF00FF00AA001B
:00000001FF
